:020000040000FA
:020000000528D1
:080008002D2B831606309F002A
:1000100085013930860087018801890181010C142E
:1000200083121F30900050308B00A401A501A6015F
:10003000A701A3018E018F010515851488014D22AA
:100040008B17A31D2928861E2E28061E3228861DE2
:10005000472823186428A318692873282623861E96
:10006000692873282623061A73287E208420A70A6D
:100070000C3027020319A70123158B1391208B172E
:1000800023112623061A732808230823322826233F
:10009000861973287E208E018F01A4018420A50A71
:1000A0000A302502031D5A28A501A60A0630260299
:1000B0000319A60123158B13D4208B172311262394
:1000C00086197328082347287E208420142384203F
:1000D0006B287E2084200823082308238B1391207B
:1000E000D4203E228B178617A301A80803197B286A
:1000F000A8030319880163000000212880308800CC
:1001000086130430A80008006030A200881603237C
:10011000032303238812032303230323A20B86282C
:1001200008002708031D96284621D3282708013CEC
:10013000031D9C284E21D3282708023C031DA2281A
:100140005621D3282708033C031DA8285E21D32865
:100150002708043C031DAE286621D3282708053C48
:10016000031DB4286E21D3282708063C031DBA2896
:100170007621D3282708073C031DC0287E21D328D9
:100180002708083C031DC6288621D3282708093CD8
:10019000031DCC288E21D32827080A3C031DD22812
:1001A0009621D3289E2108002508031DF62826083D
:1001B000031DDC28462245292608013C031DE228B0
:1001C000A62145292608023C031DE828AE21452921
:1001D0002608033C031DEE28B62145292608043CC9
:1001E000031DF428BE214529C62145292608031DE3
:1001F000FA2814292608013C031D0029CE211429C0
:100200002608023C031D0629D62114292608033C92
:10021000031D0C29DE2114292608043C031D122984
:10022000E6211429EE2114292508013C031D1A2971
:10023000F62145292508023C031D2029FE214529D8
:100240002508033C031D2629062245292508043CD0
:10025000031D2C290E2245292508053C031D3229A2
:10026000162245292508063C031D38291E2245294A
:100270002508073C031D3E29262245292508083C60
:10028000031D44292E224529362208000030AB00E8
:100290000030AC000030AD007D2208000030AB0023
:1002A0001130AC00D030AD007D2208000030AB0032
:1002B0001F30AC00F030AD007D2208000030AB00F4
:1002C0002930AC007030AD007D2208000030AB005A
:1002D0003730AC00F030AD007D2208000030AB00BC
:1002E0004230AC00D030AD007D2208000030AB00C1
:1002F0004D30AC001030AD007D2208000030AB0066
:100300005B30AC00A030AD007D2208000030AB00B7
:100310006A30AC00D030AD007D2208000030AB0068
:100320007A30AC006030AD007D2208000030AB00B8
:100330008330AC004030AD007D2208000030AB00BF
:100340008F30AC000030AD007D2208000030AB00E3
:10035000A530AC001030AD007D2208000030AB00AD
:10036000B530AC00A030AD007D2208000030AB00FD
:10037000C930AC004030AD007D2208000030AB0039
:10038000E230AC00D030AD007D2208000230AB007E
:100390000030AC000030AD007D2208000230AB0020
:1003A0001130AC00B030AD007D2208000230AB004F
:1003B0001830AC00F030AD007D2208000230AB00F8
:1003C0002530AC007030AD007D2208000230AB005B
:1003D0003430AC009030AD007D2208000230AB001C
:1003E0004430AC002030AD007D2208000230AB006C
:1003F0004F30AC009030AD007D2208000230AB00E1
:100400006030AC00D030AD007D2208000230AB007F
:100410006D30AC002030AD007D2208000230AB0012
:100420008130AC009030AD007D2208000230AB007E
:100430009030AC008030AD007D2208000230AB006F
:10044000A030AC005030AD007D2208000230AB007F
:10045000B330AC005030AD007D2208000230AB005C
:10046000C130AC003030AD007D2208000230AB005E
:10047000D130AC000030AD007D2208000230AB006E
:10048000DF30AC007030AD007D220800231D4C2A07
:1004900008230823082308230800861A7C2A861EBE
:1004A0004F2A7E20082384201423842008234621F9
:1004B0004E2156215E2166216E2176217E218621E4
:1004C0008E2196219E21A621AE21B621BE21C621D4
:1004D000CE21D621DE21E621EE21F621FE210622C3
:1004E0000E2216221E2226222E2236223E220823E9
:1004F00008238420142384200800EA22AF22F32258
:10050000A0302B04B000BD22F3222C08B000BD2285
:10051000F3222D08B000BD22F322AF22F322A13036
:100520002B04B000BD22F3222E15C8222F09031977
:10053000AA2A29088800AA012F080310A90703186E
:100540002A14A90C2A18A9172123290888002F0882
:10055000A900942A2E11C822F322B722080085147C
:10056000F322EE220511F3228510EA220800EE2282
:1005700005118514F322EA2208000830B1002E1478
:10058000B01F2E10D722B00DB10BBF2AE1220800F8
:10059000AF010830B1000310AF0DE122AE182F14E7
:1005A000B10BCC2A2E142E192E10D722080085103C
:1005B0002E18DC2AEE2205118514F3228510EA227A
:1005C00008008510EA22AE148514F322051DAE1032
:1005D000851008008316051583120800831605117F
:1005E000831205150800F42AF52AF62AF72AF82AB4
:1005F000F92AFA2AFB2AFC2AFD2AFE2AFF2A002BC6
:10060000012B022B0800A630A000A00B052B080030
:10061000F830A10003230323A10B0A2BF830A1001B
:1006200003230323A10B102BF830A1000323032382
:10063000A10B162BF830A10003230323A10B1C2BC5
:1006400008001730A000A00B232B08006330A10086
:1006500003230323A10B282B0800F0000308F1005B
:100660000C18352B8B10A315532B0C10A40A0F302C
:100670002402031D532BA401A50A0A302502031DE1
:10068000532BA501A60A033026020319A314063032
:100690002602031D532BA601A70A23140C302702A0
:1006A000031D532BA70171088300F00E700E090083
:02400E00323F3F
:00000001FF
